:1000000023C63DC63CC63BC63AC639C638C637C607
:1000100036C674CB34C633C632C631C6DBCB2FC628
:100020002EC6000000000000000000000000007E5E
:10003000C381A581BD99C37E0000007EFFFFDBFF69
:10004000C3E7FF7E0000000044EEFEFEFE7C381099
:1000500000000010387CFEFE7C3810000000001804
:100060003C3CFFE7E718187E000000183C7EFFFFCD
:100070007E18187E00000000000000000000000054
:100080000000000000000000000000000000000070
:100090000000000000000000000000000000000060
:1000A000000000000000003E0E3A72F8CCCCCC7884
:1000B0000000003C6666663C187E181800000000D0
:1000C00000000000000000000000007F637F636309
:1000D0006367E7E6C000000018DB7EE7E77EDB1819
:1000E00000000080C0E0F8FEF8E0C08000000002E0
:1000F000060E3EFE3E0E0602000000183C7E18185A
:10010000187E3C180000006666666666000066663B
:100110000000007FDBDBDB7B1B1B1B1B0000007E6A
:1001200063303C66663C0CC67E00000000000000A8
:1001300000FEFEFE000000183C7E1818187E3C18D9
:100140007E0000183C7E18181818181800000018B7
:1001500018181818187E3C180000000000180CFE33
:100160000C18000000000000003060FE603000004D
:10017000000000000000C0C0C0FE00000000000041
:10018000002466FF662400000000000010103838CC
:100190007C7CFEFE00000000FEFE7C7C38381010E7
:1001A000000000000000000000000000000000301F
:1001B00078787830300030300000006666662400C1
:1001C000000000000000006C6CFE6C6C6CFE6C6C3F
:1001D000000030307CC0C0780C0CF83030000000DB
:1001E00000C4CC183060CC8C00000070D8D870FAF5
:1001F000DECCDC7600000030303060000000000013
:100200000000000C183060606030180C00000060C6
:1002100030180C0C0C1830600000000000663CFF29
:100220003C660000000000000018187E181800004E
:1002300000000000000000000000383860000000EE
:10024000000000FE000000000000000000000000B0
:10025000000038380000000002060C183060C08032
:100260000000007CC6CEDED6F6E6C67C000000109C
:1002700030F03030303030FC00000078CCCC0C183E
:100280003060CCFC00000078CC0C0C380C0CCC7826
:100290000000000C1C3C6CCCFE0C0C1E000000FC92
:1002A000C0C0C0F80C0CCC780000003860C0C0F8AA
:1002B000CCCCCC78000000FEC6C6060C183030301E
:1002C00000000078CCCCCC78CCCCCC780000007886
:1002D000CCCCCC7C181830700000000000383800FE
:1002E00000383800000000000038380000383818A6
:1002F0003000000C183060C06030180C00000000A6
:1003000000007E007E0000000000006030180C0637
:100310000C18306000000078CC0C18303000303001
:100320000000007CC6C6DEDEDEC0C07C00000030FF
:1003300078CCCCCCFCCCCCCC000000FC6666667CD7
:10034000666666FC0000003C66C6C0C0C0C6663C6F
:10035000000000F86C66666666666CF8000000FED9
:100360006260647C646062FE000000FE6662647C21
:10037000646060F00000003C66C6C0C0CEC6663E49
:10038000000000CCCCCCCCFCCCCCCCCC0000007899
:1003900030303030303030780000001E0C0C0C0C47
:1003A000CCCCCC78000000E6666C6C786C6C66E6B1
:1003B000000000F060606060626666FE000000C6DB
:1003C000EEFEFED6C6C6C6C6000000C6C6E6F6FEEF
:1003D000DECEC6C6000000386CC6C6C6C6C66C38BF
:1003E000000000FC6666667C606060F0000000381B
:1003F0006CC6C6C6CEDE7C0C1E0000FC6666667C43
:100400006C6666E600000078CCCCC07018CCCC7866
:10041000000000FCB430303030303078000000CCC8
:10042000CCCCCCCCCCCCCC78000000CCCCCCCCCCC4
:10043000CCCC7830000000C6C6C6C6D6D66C6C6C74
:10044000000000CCCCCC783078CCCCCC000000CCF8
:10045000CCCCCC7830303078000000FECE9818300C
:100460006062C6FE0000003C303030303030303C3E
:100470000000000080C06030180C06020000003C44
:100480000C0C0C0C0C0C0C3C000010386CC6000062
:10049000000000000000000000000000000000005C
:1004A000FF003030180000000000000000000000D5
:1004B0000000780C7CCCCC76000000E060607C66AC
:1004C000666666DC00000000000078CCC0C0CC7816
:1004D0000000001C0C0C7CCCCCCCCC7600000000C6
:1004E000000078CCFCC0CC78000000386C6060F86C
:1004F000606060F000000000000076CCCCCC7C0C8A
:10050000CC7800E060606C76666666E600000018F5
:10051000180078181818187E0000000C0C003C0C0D
:100520000C0C0CCCCC7800E06060666C786C66E6F5
:1005300000000078181818181818187E000000001D
:100540000000FCD6D6D6D6C6000000000000F8CCCD
:10055000CCCCCCCC00000000000078CCCCCCCC784B
:10056000000000000000DC666666667C60F000004B
:10057000000076CCCCCCCC7C0C1E00000000EC6ED5
:10058000766060F000000000000078CC6018CC7845
:10059000000000002060FC6060606C38000000001B
:1005A0000000CCCCCCCCCC76000000000000CCCC41
:1005B000CCCC7830000000000000C6C6D6D66C6CEB
:1005C000000000000000C66C38386CC60000000057
:1005D0000000666666663C0C18F000000000FC8CAB
:1005E0001860C4FC0000001C303060C06030301C5B
:1005F000000000181818180018181818000000E05B
:100600003030180C183030E000000073DACE0000F3
:1006100000000000000000000010386CC6C6FE009C
:1006200000000078CCCCC0C0C0CCCC78306000CC0E
:10063000CC00CCCCCCCCCC7600000C18300078CCE4
:10064000FCC0CC7800003078CC00780C7CCCCC7628
:10065000000000CCCC00780C7CCCCC760000C060D4
:100660003000780C7CCCCC760000386C6C38F80C00
:100670007CCCCC7600000000000078CCC0C0CC78E8
:1006800030603078CC0078CCFCC0C07C000000CC5E
:10069000CC0078CCFCC0C07C0000C060300078CCBE
:1006A000FCC0C07C0000006C6C0078181818187E24
:1006B000000010386C0078181818187E00006030A0
:1006C000180078181818187E000000CC003078CC7C
:1006D000CCFCCCCC000078CCCC7878CCCCFCCCCC8E
:1006E00000000C1800FCC4C0F8C0C4FC00000000EE
:1006F0000000FE1B7FD8D8EF0000003E78D8D8FE5F
:10070000D8D8D8DE00003078CC0078CCCCCCCC78EF
:10071000000000CCCC0078CCCCCCCC780000C06001
:10072000300078CCCCCCCC7800003078CC00CCCC6D
:10073000CCCCCC760000C0603000CCCCCCCCCC761D
:10074000000000666600666666663C0C18F000CC29
:100750000078CCCCCCCCCC780000CC00CCCCCCCCB1
:10076000CCCCCC7800000000000078CCDCECCC785D
:1007700000003C66606060FC6060C0FE0000003A03
:100780006CCED6D6D6E66CB800000000000000C6DD
:100790006C386CC600000E1B18187E181818D8701C
:1007A00000000C183000780C7CCCCC7600000C18C3
:1007B000300078181818187E00000C18300078CC1B
:1007C000CCCCCC7800000C183000CCCCCCCCCC7687
:1007D00000000076DC00F8CCCCCCCCCC000076DC81
:1007E00000C6E6F6DECEC6C600000078CCCC7E00A1
:1007F000FE00000000000078CCCC7800FE00000075
:100800000000003030003060C0C0CC7800000038FC
:1008100044BAAABAB2AA443800000000000000FCA2
:100820000C0C0C0000000062E66C78306EC3860C85
:100830001F000063E66C78376FDBB33F03000030C6
:1008400030003030787878300000000000003366E7
:10085000CCCC6633000000000000CC66333366CC9D
:10086000000024924924924924924924924955AA8D
:1008700055AA55AA55AA55AA55AA6DDBB66DDBB681
:100880006DDBB66DDBB6181818181818181818187C
:1008900018181818181818F81818181818180C1804
:1008A000003078CCCCFCCCCC000078CC003078CCBC
:1008B000CCFCCCCC00006030003078CCCCFCCCCC74
:1008C0000000003844BAA2A2A2BA4438000066660A
:1008D0006666E60606E66666666666666666666678
:1008E00066666666666600000000FE0606E66666E8
:1008F000666666666666E60606FE00000000003074
:100900003078CCC0C0CC78303000CCCCCCCC78FCAB
:1009100030FC303000000000000000F818181818F3
:10092000181818181818181F0000000000001818D0
:10093000181818FF0000000000000000000000FF71
:1009400018181818181818181818181F1818181820
:1009500018180000000000FF000000000000181838
:10096000181818FF1818181818180076DC00780CDA
:100970007CCCCC76000076DC003078CCCCFCCCCCC7
:100980000000666666666760607F00000000000029
:1009900000007F6060676666666666666666E7009A
:1009A00000FF0000000000000000FF0000E7666696
:1009B00066666666666667606067666666660000AD
:1009C0000000FF0000FF0000000066666666E700AA
:1009D00000E7666666660000000000C67C6C7CC6A8
:1009E0000000CC30D80C067EC6C6C67C000000F8DD
:1009F0006C6666F666666CF8000078CC00FCC4C0D5
:100A0000F8C0C4FC000000CC00FCC4C0F8C0C4FCAA
:100A10000000603000FCC4C0F8C0C4FC000000F05E
:100A2000303030FC0000000000001830007830301A
:100A300030303078000078CC00783030303030788A
:100A4000000000CC007830303030307800001818CA
:100A5000181818F800000000000000000000001F37
:100A6000181818181818FFFFFFFFFFFFFFFFFFFF00
:100A7000FFFF000000000000FFFFFFFFFFFF001866
:100A80001818180018181818000060300078303056
:100A9000303030780000FFFFFFFFFFFF0000000054
:100AA000000018300078CCCCCCCCCC78000000789A
:100AB000CCCCD8CCCCCCF8C0600078CC0078CCCCF6
:100AC000CCCCCC78000060300078CCCCCCCCCC78CE
:100AD00000000076DC0078CCCCCCCC78000076DC52
:100AE0000078CCCCCCCCCC7800000000000066664E
:100AF0006666667B60C00000E0607C66667C60F0D5
:100B0000000000F0607C6666667C60F000001830D3
:100B100000CCCCCCCCCCCC78000078CC00CCCCCCED
:100B2000CCCCCC780000603000CCCCCCCCCCCC7819
:100B30000000060C1800666666663C0C18F018305B
:100B400000CCCCCC78303078000000FC00000000F5
:100B50000000000000000C18300000000000000041
:100B600000000000000000FC000000000000000089
:100B70003030FC303000FC0000000000000000F8C5
:100B80000000F8000000E033663CF8376FDBB33F4D
:100B90000300007FDBDBDB7B1B1B1B1B0000007EDD
:100BA00063303C66663C0CC67E000000303000FCC2
:100BB00000303000000000000000000000000000D5
:100BC0003070003C6666663C00000000000000CC0F
:100BD00000000000000000000000000000000018FD
:100BE000000000000000003070303078000000008D
:100BF000000000780C380C7800000000000000783D
:100C00000C18307C000000000000000000FCFCFC20
:100C1000FCFCFC00000000000000000000000000E0
:100C20000000B82062792042656E6564696B7400CB
:100C300033323078323430204C434420436F6E746A
:100C4000726F6C6C6572000011241FBECFE5D2E09C
:100C5000DEBFCDBF10E0A0E6B0E0EAEAF9E102C0F5
:100C600005900D92A236B107D9F711E0A2E6B0E0E7
:100C700001C01D92A93EB107E1F702D095C6C0C9D7
:100C80002F923F925F926F927F928F929F92AF923C
:100C9000BF92CF92DF92EF92FF920F931F93CF9369
:100CA000DF93CDB7DEB72A970FB6F894DEBF0FBE3D
:100CB000CDBF1A8219821C821B821E821D82188659
:100CC0001F821A86198683E082BB9FEF97BB8EEF47
:100CD00081BB96B99BBB95BBA0D483E390E03FD585
:100CE000772488249924BFEF5B2E66244AD5482FA9
:100CF000803208F067C0813009F45CC0823009F4AA
:100D000077C0833009F476C0883009F475C0893023
:100D100009F49AC08A3009F48FC08B3009F472C08C
:100D20008C3009F49EC08D3009F445C08E3009F432
:100D30009DC08F3009F49CC0803109F4A8C0813176
:100D400009F4D3C0823109F4EBC0833109F400C146
:100D5000853109F411C1863109F486C0893109F45D
:100D600010C18C3109F480C08D3109F423C18E315A
:100D700009F0BCCF06D5882309F036C102D5482F2B
:100D8000C401969587959695879596958795062D96
:100D9000252D672D3DD188E090E0880E991E90E4C6
:100DA000891691E0990608F4A1CFECE07E0EFFEEE3
:100DB000F71508F4772488249924E3D4482F803247
:100DC00008F499CFC4019695879596958795969541
:100DD0008795062D252D672DBFD588E090E0880EDC
:100DE000991E90E4891691E0990608F47FCFDDCF33
:100DF00038987CCF389A7ACF88EF9FEF880E991E6B
:100E000099206CF0C401969587959695879596954F
:100E10008795062D252D40E2672D9ED567CF94EF4F
:100E2000790EEFEEE71510F4F4EE7F2EE8E38E2E48
:100E3000E1E09E2E87E2EDCFFCE07F0E8FEE87157E
:100E400008F054CF772452CF9CD4282E9AD4382E31
:100E500098D4082F96D41127482FB801C101EFD498
:100E600045CFD0D07724A7CF8CD48BD48AD43ECF93
:100E700088D4282F853608F024E6822F9927880FFA
:100E8000991F2695820F911D99BD88BD2FCF79D4CA
:100E90008A3A09F02BCF75D4B82E73D4E82E71D4CA
:100EA000C82E6FD4F82E6DD4D82EFF2009F41ECF93
:100EB000AA24CC20A9F01B2D00E007C06E2D812FA5
:100EC000FDD40F5F1F5FC01659F05BD4482FDD20A3
:100ED000A9F76E2D812FE6D40F5F1F5FC016A9F70B
:100EE000A394E394FA1429F701CF4BD4882E9924C4
:100EF000880C991C880C991C880C991C42D49CE085
:100F0000899F702C112490E4891691E0990610F0C5
:100F100088249924EFEEE71508F0E8CE7724E6CE92
:100F200030D489832ED48A832CD4E82E2AD48B8380
:100F300028D48C8326D4C82E24D4DD24FF24082F63
:100F400096014B815C81B70189819A816ED1CECEA9
:100F500018D48D8316D48E8314D4E82E12D4D82EB0
:100F600010D4182F0ED4FF24082F212F4D2DB70198
:100F70008D819E81F5D1BACE04D4582E02D4682E2C
:100F8000B5CEFFD3E82EFF24F7E0EF22FF24EE0CCE
:100F9000FF1CEE0CFF1CEE0CFF1C89E691E0E80E36
:100FA000F91E10E0EED3F70181937F011F5F183027
:100FB000C9F79CCEE6D38F83E4D38887E2D3A82EEB
:100FC000E0D38987DED38A87DCD3C82EDAD3082F13
:100FD000D8D3DD24BB24E82E960149855A85B50176
:100FE0008F81988565D182CECCD3482FC401969548
:100FF00087959695879596958795062D252D672D2E
:10100000ABD4C9CEE0E0F4E011923097E9F708954F
:10101000BF92CF92DF92EF92FF920F931F93B82E61
:10102000162FE42EC22E8FE0E822FF24EE0CFF1CC8
:10103000EE0CFF1CEE0CFF1CE9E6F1E0EE0EFF1ECD
:10104000F70140818B2D6CD41F5F2C2DF70140815F
:10105000612F8B2D65D41F5F2C2DF7014181612FEE
:101060008B2D5ED41F5F2C2DF7014281612F8B2DBC
:1010700057D41F5F2C2DF7014281612F8B2D50D447
:101080001F5F2C2DF7014381612F8B2D49D41F5FEA
:101090002C2DF7014481612F8B2D42D41F5F2C2D05
:1010A000F7014581612F8B2D3BD41F5F2C2DF7015C
:1010B0004581612F8B2D34D41F5F2C2DF701468184
:1010C000612F8B2D2DD41F5F2C2DF7014781612FB0
:1010D0008B2D26D41F5F2C2DF7014781612F8B2D7F
:1010E0001FD41F910F91FF90EF90DF90CF90BF9092
:1010F00008953F924F925F926F927F928F929F924C
:10110000AF92BF92CF92DF92EF92FF920F931F9315
:10111000CF93DF937C014B015A016901302EA81A4D
:10112000B90AC61AD70A1A141B040CF065C061E08C
:10113000462E1C141D040CF058C041E0542E432DC3
:10114000B401C7017CD3AC14BD044CF1A114B104AB
:1011500009F459C0E601CC0FDD1F642C772467FC2D
:1011600070948701740188249924452C552447FCE8
:101170005094CC0DDD1DCA15DB0524F0CA19DB091E
:10118000E40CF51C060D171D432DB701C80157D3FC
:101190000894811C911CA814B90459F734C0C114D7
:1011A000D10489F1E501CC0FDD1F652C772467FCA4
:1011B0007094840188249924552447FC5094CA0DC6
:1011C000DB1DCC15DD0524F0CC19DD09E40CF51C84
:1011D000060D171D432DB801C70131D30894811C9A
:1011E000911CC814D90459F70EC0D094C194D108E9
:1011F000D3943FEF532EA3CFB094A194B108B394EE
:101200005FEF452E96CFDF91CF911F910F91FF9009
:10121000EF90DF90CF90BF90AF909F908F907F9096
:101220006F905F904F903F9008958F929F92AF92F2
:10123000BF92CF92DF92EF92FF920F93CF93DF9303
:101240004C015B016A0179016217730799F08417F9
:10125000950711F04EDF20C026173707C8F4E901C3
:101260007B01402FBE01C401EAD22196EC16FD0697
:10127000C0F712C04817590768F4EA016C01402F03
:10128000B501CE01DCD22196CC16DD06C0F704C034
:10129000EB01E7CFEC01F3CFDF91CF910F91FF90FE
:1012A000EF90DF90CF90BF90AF909F908F90089578
:1012B0003F924F925F926F927F928F929F92AF92E6
:1012C000BF92CF92DF92EF92FF920F931F93CF9333
:1012D000DF932C013B014A016901102F3E2C5C0178
:1012E0000894A11CB11CA416B50698F4EB01219634
:1012F000C217D30770F47A010894E108F108012FAE
:101300009E01A701BE01C50190DF2196CC15DD0528
:10131000B0F3032D9301A401B301C20186DF96014E
:10132000A401B301C40181DF9601A201B601C40189
:101330007CDF9301A201B601C20177DFDF91CF917B
:101340001F910F91FF90EF90DF90CF90BF90AF90E3
:101350009F908F907F906F905F904F903F900895F7
:101360002F923F924F925F926F927F928F929F92B5
:10137000AF92BF92CF92DF92EF92FF920F931F93A3
:10138000CF93DF93CDB7DEB763970FB6F894DEBF88
:101390000FBECDBF9B878A877D876C874E87122FB4
:1013A0000F87842E99248815990508F4F8C06815CC
:1013B000790508F4F4C0442309F4F1C0C401880F8E
:1013C000991F23E030E0281B390B3A832983498792
:1013D000590164011C821B8286E090E09E838D830C
:1013E000798B688B1B014A845B8432012FC089850D
:1013F00081508987C82EDD248B819C818C199D09A1
:10140000880F991F880F991FEAE0F0E0AE0EBF1E0B
:10141000A80EB91E2B813C812F5F3F4F3C832B834D
:101420000894611C711C0894410851080894211CFF
:10143000311C888999890197998B888BED81FE8170
:101440003496FE83ED83C216D30678F16C857D85D4
:101450006C0D7D1D012F9B01A301C201E6DE6C8591
:101460007D856C197D099B01A301C201DEDEEA8442
:10147000FB84EC0CFD1CEA85FB85EC19FD096F0172
:101480009101A701B101CF01D0DE28893989A701D7
:10149000B901C601CADEB7FEAACF2D813E81A20ED8
:1014A000B31E3985C32EDD24B5CFCE842224332448
:1014B00026E030E038872F834A845B84AC84BD8487
:1014C00035015B8A4A8A2CC0CA948C2C9924C101AC
:1014D00088199909880F991F880F991F29813A81C6
:1014E000265F3F4F280F391F3A8329830894211C18
:1014F000311C8A899B8901969B8B8A8B0894611C7D
:10150000711C0894A108B108089441085108EF81A2
:10151000F8853496F887EF838214930408F43FC06B
:10152000EC84FD84E80CF91C4F85B7018A899B89FE
:1015300086D10A851B85080D191D4F85B301C80189
:101540007ED14F85B501C8017AD10C851D8508195A
:1015500019094F85B8018A899B8971D14F85B801D6
:10156000C2016DD10A851B85081919094F85B5017E
:10157000C80165D14F85B301C80161D14F85B7015D
:10158000C2015DD189819A8197FF9ECFEF81F88555
:101590008E0F9F1F9A8389838C2C9924A7CF6396E3
:1015A0000FB6F894DEBF0FBECDBFDF91CF911F9174
:1015B0000F91FF90EF90DF90CF90BF90AF909F90F2
:1015C0008F907F906F905F904F903F902F900895F5
:1015D000DF92EF92FF920F931F93CF93DF93D62E5C
:1015E000FA01E22EF02E4491442379F0EF01219686
:1015F00001C0812F182F1F5F0F2D2E2D6D2DACD107
:10160000FE01219644914423A1F7DF91CF911F91D0
:101610000F91FF90EF90DF900895EF920F93F89461
:1016200088E10FB6F89481BD11BC0FBE80EC85BF78
:101630008AE090E09BBD8ABD80E890E099BD88BDBE
:1016400081E38FBD91E09EBD81E681BF8AE083BFCB
:1016500099BF7894D7DC9FEFE92E00E02FE430E0CB
:101660004DE051E06AE070E082E390E021DE00E4CA
:1016700025E430E04DE650E064E170E08CE390E07A
:1016800017DE80E4E82E2DE230E04DEB50E06FE015
:1016900070E086E990E00CDEB0E8EB2E00E82BE489
:1016A00030E04BED50E068E270E084EB90E000DE6B
:1016B000AFEFEA2E0FEF22E330E04FEE50E064E1AF
:1016C00070E088EC90E0F4DD00E02FEF40E35CE0B8
:1016D00068E78AE07DDF2FEF42E25CE06CE88FE0B4
:1016E00077DF88E190E02CE00FB6F894A89581BDF3
:1016F0000FBE21BD389A0F91EF9008951F920F925F
:101700000FB60F9211248F939F93EF93FF939CB189
:10171000E0916201EF5F80916301E817B9F0E09317
:101720006201FF27EE59FF4F9083809164019091F1
:101730006501019690936501809364018091640135
:1017400090916501813C910508F0929AFF91EF918B
:101750009F918F910F900FBE0F901F901895109230
:1017600062011092630192981092650110926401D7
:10177000292F332720BD89B980E98AB986E880BD41
:10178000089590916201809163019817D1F3E091DF
:101790006301EF5FE0936301F8948091640190919D
:1017A00065010197909365018093640180916401C4
:1017B00090916501803C910508F492987894FF27F8
:1017C000EE59FF4F8081992708958091640190918F
:1017D000650108950F930FB70F93959AAF93BF9339
:1017E0002F93959820916801223010F0A0E801C055
:1017F000A0E0B0916701B39524E194980D910D910B
:101800000D910D912A95D1F7B43069F4949AA89569
:10181000209168012395233020F02227209368012E
:1018200002C020936801B43F08F0B3E0B0936701B1
:101830002F91BF91AF910F910FBF0F91189521E09C
:101840008034920770F5603F60F5582F577030E88C
:10185000503019F036955A95E9F7969587959695F3
:101860008795A82FB62FBC5FF894939A5C919398B4
:10187000789447FF03C0532B5C9304C030955323E7
:101880005C933095A068F894939A5C9193987894BF
:1018900046FF03C0532B5C9304C0309553235C93E5
:1018A00030950895883248F4603F38F4A82FAA0F85
:1018B000B62FBC5F4C93A0684C930895803578F5A3
:1018C000603F68F5A82FB62FBC5F55276627441FD9
:1018D000551F441F661F441F551F441F661F441F8A
:1018E000551F441F661F441F551F441F661F70EF7E
:1018F000A0FF7295A0FF5295F894939A4C919398FB
:1019000078944723542B5C93A0FF6295A068F894C9
:10191000939A4C91939878944723642B6C930895F1
:101920008832C8F4603FB8F4880FB62FBC5F902FA0
:101930009223202B642FA82F07FD409527FF4427D3
:1019400097FD4FEF4C93A06806FD609526FF662734
:1019500096FD6FEF6C930895883228F5603F18F577
:10196000E42FFCE0EF9FF001EE5DFF4F5CE0880F9D
:10197000B62FBC5F902F9223202B4591642FA82F68
:1019800007FD409527FF442797FD4FEF4C93A06834
:1019900006FD609526FF662796FD6FEF6C93B39565
:0A19A0005A9559F711240895FFCF5E
:0219AA00000437
:00000001FF
